:020000040000FA
:060000003CEF10F01200BD
:020006001200E6
:0600080015EF01F01200EB
:02000E000100EF
:0C0010009420000000010000C40000006B
:04001C00D9CFE6FF53
:10002000E1CFD9FFFB0EDBCF1DF0FC0EDBCF1EF0C6
:10003000FD0EDBCF1FF0FE0EDBCF20F02034000ED4
:10004000201809E6D880000E1D54000E1E54000E24
:100050001F54000E20540CE2D950FB0FE96EFF0E26
:10006000DA20EA6EEE06000EEE5AEE5AEE5ADAD7B3
:10007000E552E7CFD9FF1200948E949C200EAF6E0C
:10008000AC8AAC84AC98AC9CAB8EAB9CAB889E9895
:100090009E9A9D8AF28EF28C1200D9CFE6FFE1CFB4
:1000A000D9FFE65200018751851902E1885186196E
:1000B00001E1F8D785C0E9FF86C0EAFF852B000E75
:1000C0008623EFCFDFFF9C0E855D010E865904E38A
:1000D0005C0E856F010E866FDF5000D0E552E55251
:1000E000E7CFD9FF1200D9CFE6FFE1CFD9FF020E4B
:1000F000E126DE6ADD6AACB210D0DF2A010E01E330
:10010000DB2AD9CFE9FFDACFEAFF100ED880EE5410
:10011000270EED5401E206D0EED7FE0EDB50AD6E99
:100120009EA8FED7020EE15C02E2E16AE552E16EB2
:10013000E552E7CFD9FF1200D9CFE6FFE1CFD9FFD3
:10014000030EE126FD0EDBCFDEFFDBCFDDFFA5DFFB
:10015000E76E020EE7CFDBFFFC0EDB50F36E020E04
:10016000DB50F35C0DE0FD0EDBCFE9FFDB2AFE0E7A
:10017000DBCFEAFF01E3DB2A020EDBCFEFFFE7D79D
:10018000FD0EDBCFE9FFFE0EDBCFEAFFEF6ADECF2D
:1001900000F0DDCF01F000C0F3FF01C0F4FF030E5B
:1001A000E15C03E200D0E16AE552E16EE552E7CF9F
:1001B000D9FF1200D9CFE6FFE1CFD9FF020EE12629
:1001C000DE6ADD6AFD0EDBCFE9FFFE0EDBCFEAFF64
:1001D000EF5014E0FD0EDBCFE9FFFE0EDBCFEAFFB0
:1001E000EF50E66E80DFE552DF2A010E01E3DB2AE5
:1001F000FD0EDB2AFE0E01E3DB2AE4D7010EF36ECF
:10020000F46A020EE15C03E200D0E16AE552E16EBD
:10021000E552E7CFD9FF12000D0EE66E64DFE5521E
:100220000A0EE66E60DFE5521200DACFE4FFE2CF9D
:10023000DAFFE9CFE4FFEACFE4FFF6CFE4FFF7CF40
:10024000E4FFF5CFE4FFF3CFE4FFF4CFE4FFFACF10
:10025000E4FF00EE18F0140EE80403E3EECFE4FF31
:10026000FBD700EE00F0180EE80403E3EECFE4FF46
:10027000FBD7E6529EAA4DD0DAEC0FF00001D96F01
:10028000AB50040B03E1AB50020B02E0AB98AB8820
:10029000ACA2FED781B205D0D9C0E6FF15EC10F0B4
:1002A000E552080E0001D95D0DE1000EE76ED81988
:1002B000E8AE02D0D83503D0E750D880D85501E257
:1002C000D80727D00D0ED95D17E0400EE76ED8197C
:1002D000E8AE02D0E73402D0E750D85D0DE2D85145
:1002E000D82BE96EEA6AE9BEEA685C0EE926010EDF
:1002F000EA22D9C0EFFF0DD0D8C0E9FFEA6AE9BE13
:10030000EA685C0EE926010EEA22EF6AD86B010E5C
:10031000846F9EA413D00101C25107E1BECFCCF07F
:10032000BFCFCDF0010EC26F08D0CD80BECFCEF0D2
:10033000BFCFCFF0010EC36FC26B9E94E55200EEAB
:1003400017F0180EE80403E3E5CFEDFFFBD700EE4E
:100350002BF0140EE80403E3E5CFEDFFFBD7E5CF68
:10036000FAFFE5CFF4FFE5CFF3FFE5CFF5FFE5CFEB
:10037000F7FFE5CFF6FFE5CFEAFFE5CFE9FFE5CFF1
:10038000DAFF1100D9CFE6FFE1CFD9FF0A0EE1264F
:1003900000014B0E826F010E836FFC0EDBCF00F06D
:1003A000010EE76E0018E8AE02D0003403D0E7502B
:1003B000D880005401E2DBD0FC0EDB5028E1FD0EBA
:1003C000DBCF00F0FE0EDBCF01F0060E00C0DBFF3E
:1003D000070E01C0DBFF080EDB6A090EDB6A82C074
:1003E000E6FF83C0E6FFD950060FE96EDACFEAFFD9
:1003F000EECFE6FFEECFE6FFEECFE6FFEFCFE6FF74
:10040000E2EC0DF0006E060EE15E005010D082C0EE
:10041000E6FF83C0E6FFFD0EDBCFE6FFFE0EDBCF7F
:10042000E6FF48EC0DF0E552E552E552E5520001D9
:1004300097AD84D04B0EE66E010EE66ECCEC0FF05D
:10044000E552E552020EF3CFDBFF030EF4CFDBFFE4
:10045000DE6ADD6ADECF00F0DDCF01F0020EDBCF19
:1004600002F0030EDBCF03F00250005C0350015892
:100470002EE2020EDBCF02F0030EDBCF03F0DE50E4
:10048000025CE96EDD500358EA6EE906000EEA5A96
:100490004B0EE926010EEA22EF50E66EFC0EDB5011
:1004A000040F006E016A00BE0168DE50005CE96E58
:1004B000DD500158EA6E4B0EE926010EEA22E552A4
:1004C000E750EF6EDF2A010E01E3DB2AC3D7DE6AB5
:1004D000DD6ADECF00F0DDCF01F0FC0EDB50050F52
:1004E000046E056A04BE0568020EDB50045C026EF1
:1004F000030EDB500558036E0250005C0350015898
:100500001DE2000197A90BD0DECFE9FFDDCFEAFFA6
:100510004B0EE926010EEA22300EEF6E0AD0DECF36
:10052000E9FFDDCFEAFF4B0EE926010EEA22200E9D
:10053000EF6EDF2A010E01E3DB2ACBD7FC0EDB5086
:10054000050FE96EEA6AE9BEEA684B0EE926010E7C
:10055000EA22EF6A82C0E6FF83C0E6FF2BDEE552A7
:10056000E552020EF3CFDBFF030EF4CFDBFF0A0EE2
:10057000E15C02E2E16AE552E16EE552E7CFD9FFC4
:100580001200D9CFE6FFE1CFD9FF0E0EE126F90E1A
:10059000DBCFDEFFDBCFDDFFF80EDBCF02F0000E9E
:1005A000E76E0218E8AE02D0023403D0E750D880DC
:1005B000025402E3070E12D0F80EDBCF03F0160E42
:1005C000E76E0318E8AE02D0033403D0E750D880BA
:1005D000035402E2170E02D0F80EDB28006E016A07
:1005E00000BE0168080E00C0DBFF090E01C0DBFF82
:1005F000020EDB6A030EDB6AFB0EDBCF00F0FC0EA3
:10060000DBCF01F0FD0EDBCF02F0FE0EDBCF03F0FF
:10061000226A236A246A256A00C01DF001C01EF008
:1006200002C01FF003C020F064EC0CF0010A33E1BB
:10063000F90EDBCFE9FFDB2AFA0EDBCFEAFF01E39D
:10064000DB2A2D0EEF6EFB0EDBCF00F0FC0EDBCFB6
:1006500001F0FD0EDBCF02F0FE0EDBCF03F0226ACD
:10066000236A800E246EBF0E256E00C01DF001C0EF
:100670001EF002C01FF003C020F088EC0BF0FB0E50
:100680001DC0DBFFFC0E1EC0DBFFFD0E1FC0DBFF2D
:10069000FE0E20C0DBFFFB0EDBCF00F0FC0EDBCF3D
:1006A00001F0FD0EDBCF02F0FE0EDBCF03F0226A7D
:1006B000236A246A256A00C01DF001C01EF002C032
:1006C0001FF003C020F05BEC0CF0010A4AE1FB0EC6
:1006D000DBCF00F0FC0EDBCF01F0FD0EDBCF02F034
:1006E000FE0EDBCF03F0226A236A800E246E3F0EDB
:1006F000256E00C01DF001C01EF002C01FF003C037
:1007000020F064EC0CF0010A2CE1006A016A200E72
:10071000026E410E036ED950FB0FE96EFF0EDA2018
:10072000EA6EEECF1DF0EECF1EF0EECF1FF0EFCF52
:1007300020F000C022F001C023F002C024F003C06A
:1007400025F088EC0BF020C0EDFF1FC0EDFF1EC0B0
:10075000EDFF1DC0EFFF020EDB06030E01E2DB061C
:10076000B6D7FB0EDBCF00F0FC0EDBCF01F0FD0EA9
:10077000DBCF02F0FE0EDBCF03F0226A236A200EED
:10078000246E410E256E00C01DF001C01EF002C097
:100790001FF003C020F064EC0CF0010A2EE0FB0E09
:1007A000DBCF00F0FC0EDBCF01F0FD0EDBCF02F063
:1007B000FE0EDBCF03F0226A236A200E246E410E68
:1007C000256E00C01DF001C01EF002C01FF003C066
:1007D00020F035EC0BF0FB0E1DC0DBFFFC0E1EC045
:1007E000DBFFFD0E1FC0DBFFFE0E20C0DBFF020E95
:1007F000DB2A030E01E3DB2AB4D7020EDBCF00F0C5
:10080000030EDBCF01F0D950080FE96EDACFEAFF13
:100810000050EE260150ED22010EF36E040EF3CFD0
:10082000DBFF050EDB6A040EDBCF1EF0050EDBCF0F
:100830001FF070EC0AF00A0E1DC0DBFF0B0E1EC08D
:10084000DBFF0C0E1FC0DBFF0D0E20C0DBFF040E14
:10085000DBCF00F0050EDBCF01F0080EDBCF02F09E
:10086000090EDBCF03F001500318E8AE02D00334C9
:1008700004D00250005C035001582EE20A0EDBCF78
:1008800000F00B0EDBCF01F00C0EDBCF02F00D0EF3
:10089000DBCF03F0226A236A200E246E410E256E00
:1008A00000C01DF001C01EF002C01FF003C020F008
:1008B00035EC0BF00A0E1DC0DBFF0B0E1EC0DBFF7C
:1008C0000C0E1FC0DBFF0D0E20C0DBFF040EDB2A69
:1008D000050E01E3DB2ABBD70A0EDBCF04F00B0EBB
:1008E000DBCF05F00C0EDBCF06F00D0EDBCF07F0F3
:1008F000226A236A246A400E256E04C01DF005C0DA
:100900001EF006C01FF007C020F035EC0BF01DC034
:1009100000F01EC001F01FC002F020C003F0D9504B
:10092000FB0FE96EFF0EDA20EA6EEECF1DF0EECF80
:100930001EF0EECF1FF0EFCF20F000C022F001C07C
:1009400023F002C024F003C025F09FEC0AF020C081
:10095000EDFF1FC0EDFF1EC0EDFF1DC0EFFFFB0E42
:10096000DBCF00F0FC0EDBCF01F0FD0EDBCF02F0A1
:10097000FE0EDBCF03F0226A236A200E246E410EA6
:10098000256E00C01DF001C01EF002C01FF003C0A4
:1009900020F064EC0CF0010A13E0FB0EDB6AFC0EA5
:1009A000DB6A800EF36EFD0EF3CFDBFF3F0EF36EBE
:1009B000FE0EF3CFDBFF020EDB2A030E01E3DB2A80
:1009C000020EDBCF00F0030EDBCF01F00001800E42
:1009D00001145FE0F90EDBCFE9FFDB2AFA0EDBCF73
:1009E000EAFF01E3DB2A300EEF6EF90EDBCFE9FF01
:1009F000DB2AFA0EDBCFEAFF01E3DB2A2E0EEF6ED5
:100A0000080EDBCF00F0090EDBCF01F0800E0114E1
:100A100014E0020EDBCF02F0030EDBCF03F0080E72
:100A2000DB50025C006E090EDB500358016E020EB3
:100A300000C0DBFF030E01C0DBFF040EDB68050E08
:100A4000DB68040EDBCF00F0050EDBCF01F0020EF9
:100A5000DBCF02F0030EDBCF03F003500118E8AE4A
:100A600002D0013404D00050025C0150035811E25E
:100A7000F90EDBCFE9FFDB2AFA0EDBCFEAFF01E359
:100A8000DB2A300EEF6E040EDB06050E01E2DB06FC
:100A9000D8D7040EDB6A050EDB6A040EDBCF00F04C
:100AA000050EDBCF01F0080EDBCF02F0090EDBCF25
:100AB00003F001500318E8AE02D0033404D0025012
:100AC000005C0350015801E3ACD0FB0EDBCF1DF0FE
:100AD000FC0EDBCF1EF0FD0EDBCF1FF0FE0EDBCFDA
:100AE00020F0F5EC0BF0060E1EC0DBFF070E1FC05A
:100AF000DBFF300EE76E060EDBCF00F0070EDBCF1C
:100B000001F0E7500026000E0122F90EDBCFE9FFCD
:100B1000DB2AFA0EDBCFEAFF01E3DB2A00C0EFFF9E
:100B2000040EDBCF00F0050EDBCF01F0020EDB5030
:100B3000001803E1030EDB5001180BE1F90EDBCFC7
:100B4000E9FFDB2AFA0EDBCFEAFF01E3DB2A2E0EF8
:100B5000EF6E060EDBCF1EF0070EDBCF1FF070EC42
:100B60000AF00A0E1DC0DBFF0B0E1EC0DBFF0C0ED1
:100B70001FC0DBFF0D0E20C0DBFF1DC000F01EC03C
:100B800001F01FC002F020C003F0D950FB0FE96E46
:100B9000FF0EDA20EA6EEECF1DF0EECF1EF0EECFA4
:100BA0001FF0EFCF20F000C022F001C023F002C000
:100BB00024F003C025F09EEC0AF020C0EDFF1FC01A
:100BC000EDFF1EC0EDFF1DC0EFFF006A016A200EA1
:100BD000026E410E036ED950FB0FE96EFF0EDA2054
:100BE000EA6EEECF1DF0EECF1EF0EECF1FF0EFCF8E
:100BF00020F000C022F001C023F002C024F003C0A6
:100C000025F088EC0BF020C0EDFF1FC0EDFF1EC0EB
:100C1000EDFF1DC0EFFF040EDB2A050E01E3DB2A0A
:100C20003CD7F90EDBCFE9FFFA0EDBCFEAFFEF6A24
:100C30000E0EE15C02E2E16AE552E16EE552E7CFB9
:100C4000D9FF1200D9CFE6FFE1CFD9FF060EE1268A
:100C50000001979DFB0EDBCF1DF0FC0EDBCF1EF0DD
:100C6000FD0EDBCF1FF0FE0EDBCF20F024EC0CF0EE
:100C70001CC0DEFF1DC0DEFF1EC0DEFF1FC0DDFF8B
:100C8000DD52DD52FB0EDBCF04F0FC0EDBCF05F0B6
:100C9000FD0EDBCF06F0FE0EDBCF07F0F90EDBCF4B
:100CA0001EF0FA0EDBCF1FF070EC0AF01DC008F04A
:100CB0001EC009F01FC00AF020C00BF008C022F0CF
:100CC00009C023F00AC024F00BC025F004C01DF0B9
:100CD00005C01EF006C01FF007C020F088EC0BF026
:100CE0001DC000F01EC001F01FC002F020C003F0C4
:100CF000F90EDBCF14F0FA0EDBCF15F0166A176A87
:100D000015AE02D01668176814C01CF015C01DF08F
:100D100016C01EF017C01FF0DFCF21F0010EDBCF91
:100D200022F0020EDBCF23F0030EDBCF24F07BECAE
:100D30000FF018C010F019C011F01AC012F01BC04B
:100D400013F010C01CF011C01DF012C01EF013C033
:100D50001FF085EC0AF01DC00CF01EC00DF01FC086
:100D60000EF020C00FF00CC022F00DC023F00EC01A
:100D700024F00FC025F000C01DF001C01EF002C01D
:100D80001FF003C020F09EEC0AF0F5EC0BF0040E0F
:100D90001EC0DBFF050E1FC0DBFF000EE66E010E5E
:100DA000E66ED9CFE9FFDACFEAFFEECFE6FFEECF6E
:100DB000E6FFEECFE6FFEFCFE6FFE2EC0DF0006ED0
:100DC000060EE15E0050000EE66E010EE66EDAECF5
:100DD00000F0E552E552F3CFA4F0F4CFA5F02E0ECB
:100DE000E66E73EC00F0E552F80EDBCFE6FFE66A44
:100DF000040EDBCFE6FF050EDBCFE6FFC2EC01F011
:100E0000E552E552E552E552060EE15C02E2E16A86
:100E1000E552E16EE552E7CFD9FF1200D9CFE6FFE8
:100E2000E1CFD9FFE652800EDF6EDF50000813E2FB
:100E3000FE0EDB50DF1406E0310EE66E73EC00F0C0
:100E4000E55205D0300EE66E73EC00F0E552DF405F
:100E50007F0BDF6EEAD7E552E552E7CFD9FF1200EC
:100E6000D9CFE6FFE1CFD9FF020EE126FE0EDB501F
:100E7000F00BE8380F0B300FDF6EDF50390803E25C
:100E8000070EDF24DF6EFE0EDB500F0B300FE76E18
:100E9000010EE7CFDBFFDB5039080AE2070E006ED8
:100EA000010EDBCFE7FF0050E726010EE7CFDBFFA7
:100EB000DFCFE6FF73EC00F0E552010EDBCFE6FF7B
:100EC00073EC00F0E552680EE66E73EC00F0E5524C
:100ED000020EE15C02E2E16AE552E16EE552E7CF23
:100EE000D9FF1200816893689380938293849386DC
:100EF0009388938A938C938EC26A070EC16E926E0A
:100F0000896A8268860E946E9490949294849496E2
:100F10009498949A949C948E1200E4DF3CEC00F038
:100F20000C0EE66E73EC00F0E552F00EE66E490E24
:100F3000E66E020EE66EE66A0EEC00F0E552E55251
:100F4000E552E5520101000E406F010E416F9EC156
:100F500000F09FC101F0026A00C0E6FF01C0E6FF99
:100F600002C0E6FF40C1E6FF41C1E6FFB3EC0FF06F
:100F7000036E050EE15E035040C1E6FF41C1E6FF8E
:100F8000DAEC00F0E552E552F3CFA4F0F4CFA5F08F
:100F9000A0C100F0A1C101F0026A00C0E6FF01C0DB
:100FA000E6FF02C0E6FF40C1E6FF41C1E6FFB3EC49
:100FB0000FF0036E050EE15E035040C1E6FF41C134
:100FC000E6FFDAEC00F0E552E552F3CFA4F0F4CFFF
:100FD000A5F0A2C100F0A3C101F0026A00C0E6FFC3
:100FE00001C0E6FF02C0E6FF40C1E6FF41C1E6FFE7
:100FF000B3EC0FF0036E050EE15E035040C1E6FF57
:1010000041C1E6FFDAEC00F0E552E552F3CFA4F07F
:10101000F4CFA5F0A00EE66E860EE66E010EE66E2B
:10102000E66A0EEC00F0E552E552E552E552CD6A73
:10103000CD8ECD9ACD980001CD0ED46FCC0ED56F4C
:101040004C0ED66F3E0ED76FCD96CD84CD92CD90FF
:101050009F80000EE66EE66AF9EC0FF0E552E5526D
:101060009E90F28C9D90F29EF29C9484B19C050E11
:10107000BD6ED08EF28E0101C26BC36B81A20CD00B
:10108000CD9ACD980001CD0ED46FCC0ED56F4C0EFD
:10109000D66F3E0ED76F0AD0CD8ACD880001CD0E17
:1010A000D46FCC0ED56FD66F3F0ED76FB26BB36BCC
:1010B000B46BB56BA26BA36BB66BB76BB86BB96B4C
:1010C000BA6B240EBB6FF40EBC6FBD6B9E9001011A
:1010D000C36BC26B0001AA6BAB6BAC6BAD6BAE6B41
:1010E000AF6BB06BB16B9E949D84CD800101C351F9
:1010F00011E19E50010B0EE0C25104E10001AC2B46
:10110000000EAD230101C20504E10001B02B000E69
:10111000B1239E900101C351E9E09D94E66AE66A1D
:10112000A2C000F0A3C001F0090ED8800056000E46
:10113000015600C0E6FF01C0E6FFC2EC01F0E55237
:10114000E552E552E552090EE66E73EC00F0E55209
:101150000101C36BCCC000F0CDC001F0001E011E28
:1011600000500001CE25CA6F0150CF21CB6F000E79
:10117000E66E010EE66ECAC000F0CBC001F0026A56
:10118000036A00C0E6FF01C0E6FF02C0E6FF03C03D
:10119000E6FFE2EC0DF0046E060EE15E0450000E78
:1011A000E66E010EE66EDAEC00F0E552E552F3CFA2
:1011B000A4F0F4CFA5F0CAC000F0CBC001F0026AE1
:1011C000036AB20EE96E000EEA6EEE5000240001D2
:1011D000B26FEE500120B36FEE500220B46FEE50AC
:1011E0000320B56F0CEC01F0100EE66E270EE66ED4
:1011F000E66AE66A0EEC00F0E552E552E552E55289
:101200000001A22B000EA3230A0EA25D000EA3591B
:1012100001E25DD7B2C01CF0B3C01DF0B4C01EF037
:10122000B5C01FF083EC0AF01DC004F01EC005F02D
:101230001FC006F020C007F0AAC01CF0ABC01DF014
:10124000ACC01EF0ADC01FF083EC0AF01DC008F06A
:101250001EC009F01FC00AF020C00BF008C022F029
:1012600009C023F00AC024F00BC025F004C01DF013
:1012700005C01EF006C01FF007C020F09FEC0AF06A
:101280001DC000F01EC001F01FC002F020C003F01E
:10129000AEC01CF0AFC01DF0B0C01EF0B1C01FF05A
:1012A00083EC0AF01DC00CF01EC00DF01FC00EF044
:1012B00020C00FF00CC022F00DC023F00EC024F0AF
:1012C0000FC025F000C01DF001C01EF002C01FF0CD
:1012D00003C020F09FEC0AF01DC0BEF01EC0BFF09E
:1012E0001FC0C0F020C0C1F02A0EE66E73EC00F003
:1012F000E552200EE66E73EC00F0E552006A240E13
:10130000016E740E026E490E036EB2C01CF0B3C0C3
:101310001DF0B4C01EF0B5C01FF083EC0AF01DC074
:1013200008F01EC009F01FC00AF020C00BF0D4C0A6
:1013300022F0D5C023F0D6C024F0D7C025F008C0D5
:101340001DF009C01EF00AC01FF00BC020F088EC91
:101350000BF01DC004F01EC005F01FC006F020C039
:1013600007F004C022F005C023F006C024F007C037
:1013700025F000C01DF001C01EF002C01FF003C028
:1013800020F035EC0BF01DC0D0F01EC0D1F01FC016
:10139000D2F020C0D3F0020EE66E40C1E6FF41C19C
:1013A000E6FFD0C0E6FFD1C0E6FFD2C0E6FFD3C063
:1013B000E6FFC1EC02F0006E070EE15E005040C196
:1013C000E6FF41C1E6FFDAEC00F0E552E552F3CF6B
:1013D000A4F0F4CFA5F0200EE66E73EC00F0E55219
:1013E000480EE66E73EC00F0E5527A0EE66E73EC92
:1013F00000F0E552090EE66E73EC00F0E552800E47
:10140000006E960E016E180E026E4B0E036ED4C067
:1014100022F0D5C023F0D6C024F0D7C025F0BEC03E
:101420001DF0BFC01EF0C0C01FF0C1C020F088EC8E
:101430000BF01DC004F01EC005F01FC006F020C058
:1014400007F004C022F005C023F006C024F007C056
:1014500025F000C01DF001C01EF002C01FF003C047
:1014600020F035EC0BF01DC0D0F01EC0D1F01FC035
:10147000D2F020C0D3F0020EE66E40C1E6FF41C1BB
:10148000E6FFD0C0E6FFD1C0E6FFD2C0E6FFD3C082
:10149000E6FFC1EC02F0006E070EE15E005040C1B5
:1014A000E6FF41C1E6FFDAEC00F0E552E552F3CF8A
:1014B000A4F0F4CFA5F0200EE66E73EC00F0E55238
:1014C000480EE66E73EC00F0E5527A0EE66E73ECB1
:0C14D00000F0E5520CEC01F0D1D5120048
:0414DC00279E08D06F
:1014E000279E1FAE05D01E6C1F1EE86A1F22278E86
:1014F0001FC019F01EC018F02B6A2A6A8E0E1A6ED1
:101500001B6ADEEF0CF0279E0CD0279E1FAE09D081
:101510001C6C1D1E1E1E1F1EE86A1D221E221F227D
:10152000278E1FC019F01EC018F01DC02BF01CC064
:101530002AF09E0E1A6E1B6ADEEF0CF0257E276ADB
:101540001AEC0DF032EC0DF027B6C2EF0CF027A22A
:101550000AD027AA03D027BEC2EF0CF027A4CEEFF3
:101560000CF0CBEF0CF027AA05D027ACCEEF0CF097
:10157000CBEF0CF027A00AD027A808D027BE04D0B4
:1015800027A402D0D7EF0CF0DBEF0CF02A6A1B6A1D
:101590002550205C296E10E31DC02BF01EC018F0F2
:1015A0001FC019F020C028F022C01DF023C01EF07B
:1015B00024C01FF0273A09D022C02BF023C018F016
:1015C00024C019F025C028F0296C279E27BC278E3F
:1015D00028C01AF027B00AEF0DF01A0E29600AEFA2
:1015E0000DF01A6A206A27A408D01D6C1E1E1F1E4B
:1015F000201EE86A1E221F22202227AC08D02B6C56
:10160000181E191E1A1EE86A182219221A221C6AAC
:10161000295207E020341F321E321D321C32292E7F
:10162000F9D71D502B261E5018221F50192220506A
:101630001A221CC02AF0279E1AAE0BD02A6C2B1E31
:10164000181E191E1A1EE86A2B22182219221A22A5
:10165000278E1AA006D0D880193218322B322A329F
:10166000282A28C01AF0DEEF0CF0276A1AEC0DF0D9
:1016700032EC0DF027B6C2EF0CF027A205D027BA46
:10168000C2EF0CF0C9EF0CF027BAD5EF0CF027A091
:1016900005D027B8C2EF0CF0D5EF0CF027B8C9EF92
:1016A0000CF01B6A7F0E20241A6EE86A1B2225505C
:1016B0001A5EE86A1B5A1A0E286E206A2A6A2B6A7A
:1016C000186A196A22501D5E23501E5A24501F5A50
:1016D000000E205A09E722501D2623501E222450B6
:1016E0001F22000E202201D02A8AD8901D361E36D5
:1016F0001F362036D8902A362B3618361936282E23
:10170000E1D71F501E101D10D8A42A8ADEEF0CF05E
:10171000276A1AEC0DF032EC0DF027B6C2EF0CF090
:1017200027A205D027B8C2EF0CF0C9EF0CF027AA0A
:1017300005D027B0C2EF0CF0C9EF0CF027B002D0F3
:1017400027A802D0D5EF0CF01B6A255020241A6E72
:10175000E86A1B227E0E1A5EE86A1B5A2A6A2B6A06
:10176000186A196A24501F02F4CF19F0F3CF18F049
:1017700023501F02F3502B26F4501822000E19227A
:1017800024501E02F3502B26F4501822000E19226A
:1017900022501F02F3502A26F4502B22000E18224A
:1017A000192223501E02F3502A26F4502B22000E39
:1017B0001822192224501D02F3502A26F4502B22FD
:1017C000000E1822192222501E02F4502A26000E62
:1017D0002B221822192223501D02F4502A26000E13
:1017E0002B2218221922DEEF0CF0276A1AEC0DF0DA
:1017F00027B6FFEF0BF027A20ED027B405D07F0E3F
:101800001F6EFF0E1E6E1FD0800E1F6E1E6A1BD035
:101810001F6A1E6A18D027B0FBD78F0E2060EDD745
:101820007E0E2064F5D78E0E205C05E0D8901F3226
:101830001E32202AF8D727A406D01E6C1F1EE86A85
:101840001F221FAEE5D71200276A1AEC0DF027B64B
:101850002EEF0CF027A20FD027B407D07F0E1F6EFB
:10186000FF0E1E6E1D6E1C6E25D0800E1F6E01D0E9
:101870001F6A000EF6D727B0FBD71C6A9F0E2060A8
:10188000EBD77E0E2064F4D79E0E205C07E0D89044
:101890001F321E321D321C32202AF6D727A40AD04E
:1018A0001C6C1D1E1E1E1F1EE86A1D221E221F22EA
:1018B0001FAEDED712006DEC0CF027B6000C27B07F
:1018C000000C27B4000C010C6DEC0CF027B6000CDA
:1018D00027B0000C27A4000C010C276A1AEC0DF0AD
:1018E00032EC0DF027B6120027AE08D027A004D0A6
:1018F00027A802D027801200279012002550205CD4
:101900000BE124501F5C08E123501E5C05E12250CE
:101910001D5C02E127801200D8A002D0278E10D0D3
:10192000205025C020F0256E1F5024C01FF0246ECB
:101930001E5023C01EF0236E1D5022C01DF0226ECB
:101940002550205C10E0FF0F09E0279027B403D05A
:1019500027AE2784120027AE27941200252AD8909C
:1019600024322332223222501D5E23501E5A24502C
:101970001F5A1FBEEAD7D8901D361E361F36202E9E
:10198000F8D7C8D77F0E206EFF0E1F6E1E6E1D6E1D
:1019900012007F0E27BEFF0E206E02D07F0E206E3B
:1019A000800E1F6E1E6A1D6AF3D727AE04D0800E0C
:1019B000206E1F6AF7D7206A1F6AF4D719501810D3
:1019C0002B102A10F8E01BBEF0D719BE0CD01A500D
:1019D0001B10EBE0D8902A362B36183619361A062B
:1019E000D8A01B06F2D71B50D4E11A28D2E02AAEA9
:1019F00011D07F0E2A1402E12BA00CD02B2AE86A0A
:101A00001822192207E3D880193218322B321A2AE9
:101A10001A28BFE01A50C9E02BC01DF018C01EF0F4
:101A200019341F6E1A30206E1F32209E27BE208E62
:101A3000C8EF0CF01F36203602E32784277E06E12C
:101A40002780206A1F6A1E6A1D6A1200202803E090
:101A5000D8801F321200D8901F3202E12782120074
:101A6000278612002436253602E3278C277E06E1DE
:101A70002788256A246A236A226A1200252803E03F
:101A8000D88024321200D8902432EAE1278A12004A
:101A9000D9CFE6FFDACFE6FFFA0EE3CFD9FFFB0E90
:101AA000E3CFDAFFFD0EE35209E72D0EDE6EFC0EEA
:101AB000E31EE32AFD0ED8B4E306E31EE652E65227
:101AC000E652FD0EE124E76EFF0EE220E46EE652E0
:101AD000F70EE3CFE6FFF70EE3CFE6FFB8EC0DF02D
:101AE000F90EE124E96EFF0EE220EA6EA8EC0DF09B
:101AF0000AE1A5EC0DF009E1A8EC0DF008E1A5EC78
:101B00000DF007E108D0B3EC0DF0AEEC0DF0B3EC46
:101B10000DF0AEEC0DF0B3EC0DF0DE6AF90EE1263F
:101B2000FF0EE222FF0EE3CFDAFFE552FF0EE3CF16
:101B3000D9FFE552FC0EE124E96EFF0EE220EA6EC9
:101B4000EECFF3FFEFCFF4FF1200EF380F0B1200D0
:101B5000EF500F0B02E1EE52D8841200EF380F0B5A
:101B6000300FDE6E1200EE500F0B300FDE6E1200E3
:101B7000FC0EE3CFE9FFFD0EE3CFEAFF100EE66EA9
:101B8000EE6AEE6AEF6AD890FD0EE336FE0EE3369B
:101B9000ED36ED36EF36FF0EE30609E0D9EC0DF039
:101BA000EE52D9EC0DF0EE52D9EC0DF0EDD7E56E1A
:101BB0001200030EEF24E8B6EF6E300EEF24E8BEFD
:101BC000EF6E000CD9CFE6FFDACFE6FFF80EE3CFD9
:101BD000D9FFF90EE3CFDAFFE652E652E652E652BB
:101BE000E652FB0EE124E76EFF0EE220E46EE652C1
:101BF000F30EE3CFE6FFF30EE3CFE6FFF30EE3CF02
:101C0000E6FFF30EE3CFE6FF67EC0EF0F50EE124FE
:101C1000E96EFF0EE220EA6E54EC0EF019E157EC8B
:101C20000EF018E154EC0EF017E157EC0EF016E14F
:101C300054EC0EF015E157EC0EF014E154EC0EF0FC
:101C400013E157EC0EF012E154EC0EF011E112D05A
:101C50005DEC0EF062EC0EF05DEC0EF062EC0EF05E
:101C60005DEC0EF062EC0EF05DEC0EF062EC0EF04E
:101C70005DEC0EF062EC0EF0DE6AF50EE126FF0E72
:101C8000E222FF0EE3CFDAFFE552FF0EE3CFD9FFEA
:101C9000E552FA0EE124E96EFF0EE220EA6EEECF85
:101CA000F3FFEFCFF4FF1200EF380F0B1200EF50ED
:101CB0000F0B02E1EE52D8841200EF380F0B300FF9
:101CC000DE6E1200EE500F0B300FDE6E1200FA0EB9
:101CD000E3CFE9FFFB0EE3CFEAFF200EE66EEE6AEC
:101CE000EE6AEE6AEE6AEF6AD890FB0EE336FC0EFF
:101CF000E336FD0EE336FE0EE336ED36ED36ED3619
:101D0000ED36EF36FF0EE3060FE096EC0EF0EE52E6
:101D100096EC0EF0EE5296EC0EF0EE5296EC0EF0C3
:101D2000EE5296EC0EF0E1D7E56E1200030EEF24B2
:0E1D3000E8B6EF6E300EEF24E8BEEF6E000C4A
:021D3E002E2E47
:101D40002E00506F727420636F6D6D203338343005
:101D500030206F7576657274200D0A00513D323067
:101D60004D687A20200D0A004331383A3138465FF9
:101D7000706572696F645F7669615F434350312EAD
:101D8000630D0A00200050524F424C454D45212022
:101D90004D657375726520494E535441424C45213F
:101DA000202B2D3525203A2000200D0A0031384601
:101DB00020506572696F646D657465722000204300
:101DC0004350312052433220202020202020002068
:101DD000204D504C4142204331382020202020000B
:101DE00020323220646563202032303131202020BF
:101DF0000020202020202020202020202020202003
:101E00002000204F766572202121212020202020D3
:101E1000202000204D6F79656E6E65203130206D79
:101E2000657320002020202020202020202020203A
:101E300020202020002054696D652045636F756C5B
:101E40006520202020002043616C69627261746902
:071E50006F6E20202020002E
:081E58000E0EF66E000EF76E8F
:101E6000000EF86E00010900F550E16F0900F55011
:101E7000E26F03E1E16701D03DD00900F550DC6F6E
:101E80000900F550DD6F0900F550DE6F090009000B
:101E9000F550E96E0900F550EA6E090009000900E5
:101EA000F550DF6F0900F550E06F09000900F6CF2B
:101EB000E3F0F7CFE4F0F8CFE5F0DCC0F6FFDDC0EB
:101EC000F7FFDEC0F8FF0001DF5302E1E05307E057
:101ED0000900F550EE6EDF07F8E2E007F9D7E3C03E
:101EE000F6FFE4C0F7FFE5C0F8FF0001E107000ED0
:061EF000E25BBFD7120007
:0A1EF6001C502102F3CF18F0F4CFC6
:101F000019F02202F3501926000EF4201A6E1C500C
:101F10002302F3501A26000EF4201B6E1C502402DC
:101F2000F3501B261D502102F3501926F4501A229B
:101F3000000E1B221D502202F3501A26F4501B22C1
:101F40001D502302F3501B261E502102F3501A2667
:101F5000F4501B221E502202F3501B261F50210258
:061F6000F3501B261200E5
:0A1F6600FB0EE3CFF6FFFC0EE3CF05
:101F7000F7FFFD0EE3CFF8FFFE0EE3CFE9FFFF0E04
:101F8000E3CFEAFFE9CFF3FFEACFF4FF0900F5CF93
:101F9000EFFFEE66FBD71200FE0EE3CFE9FFFF0E68
:101FA000E3CFEAFFF36AF46AEE5203E0F34AF42A5D
:041FB000FBD7120049
:0C1FB400D9CFE6FFDACFE6FFE1CFD9FF7E
:101FC000E2CFDAFFE652F20E0001E617ABAC03D027
:101FD000E691ABB0E681ABB4E685ABB2E687AE5036
:101FE000DF6EDF50E552E552E5CFDAFFE7CFD9FFEC
:021FF0001200DD
:0E1FF200D9CFE6FFDACFE6FFE1CFD9FFE2CF8D
:10200000DAFFE652E652FC0EDBCFDEFFDBCFDDFF70
:10201000010EDB50CF6EDF50CE6EE552E552E55239
:0A202000E5CFDAFFE7CFD9FF120089
:06202A00D9CFE6FFDACF7A
:10203000E6FFE1CFD9FFE2CFDAFFACAC04D0AC9041
:102040000001E6B3AC80FD0EDB50AD6EE552E5CF8E
:08205000DAFFE7CFD9FF12000F
:08205800000EF36E00EE00F033
:10206000060E01D81200EA6002D0EE6AFCD7F350E7
:08207000E9601200EE6AFCD7E2
:0820780015EE00F025EE00F06A
:10208000F86A279C2CEC0FF003EC00F08DEC07F0C5
:04209000FBD7120068
:0C2094003138463235325F4361706163C1
:1020A000696D5F43413535355F706F6F6C696E6781
:1020B0002E630D0A2020737472696E6720656E208E
:1020C00052414D0D00000000000000000000000023
:1020D000000000000001303030303030303000314E
:1020E0003233343536373839303132333435000411
:1020F00030303030303030303030303030303030E0
:10210000303030303030300004040404040404045F
:10211000040404040404040404040404040404047F
:10212000040404040404040404040404040404046F
:102130003E1D421D5C1D681D841D861DA91DAD1D13
:10214000BE1DCF1DE01DF11D021E131E241E351ED7
:08215000461EB315010000005A
:020000040030CA
:01000100FA04
:01000200F409
:01000300FEFE
:01000600FBFE
:00000001FF
